:050E23003238314300EC
:100D890075A40D7580FF75D44075A50C75F20F75A6
:100D9900D50175F3F075A63075B0FF75E10675E2FA
:020DA900C22264
:030E2C00020DCDE7
:020E2F00D322CC
:100CCA00C207C208E4F5D9120D89120E2F92073015
:100CDA000735120E2C7BFF7A0E7923120827EF2490
:100CEA00FF92083008107D007C06E4FFFE120D3FDB
:100CFA00E4FFFE1209ABE4FFFE0FBF00010EBE27A0
:090D0A00F8BF10F5E4F5C080FE0D
:090E1A0023213230304546550019
:0B0D130090005CEFF0FD90005BE0FF43
:050D1E00900079EDF0EA
:100D2300120DABEFC454F090007AF0900079E0FF1D
:0B0D3300120DAB90007AE02FF0E0FF03
:010D3E002292
:0B082700900067EBF0A3EAF0A3E9F0FB
:1008320090007174FFF0A3740EF0A3741AF090008C
:100842006E7401F0A37400F0A37408F090006A12B1
:100852000C9900000000E47F50FEFDFC90006AE06D
:10086200F8A3E0F9A3E0FAA3E0FBC3120C77504A25
:1008720090006AA3A3A3E0FF7BA0E4FD120B2F90DC
:10088200006EE0FBA3E475F001120C61A9F0FAEF2F
:10089200120C4F90006AE0FCA3E0FDA3E0FEA3E08F
:1008A200FFE4FAF9F8EF2401FFEA3EFEE93DFDE834
:1008B2003CFC90006A120C8D809C900071E0FBA3BE
:1008C200E0FAA3E0F9120C09FF900008E06F7062F1
:1008D200900001120C22FF900009E06F705490000A
:1008E20002120C22FF90000AE06F70469000031281
:1008F2000C22FF90000BE06F7038900004120C2263
:10090200FF90000CE06F702A900005120C22FF90FD
:10091200000DE0B5071C900006120C22FF90000E9D
:10092200E0B5070E900007120C22FF90000FE06F57
:1009320060037F0022900067E0FBA3E0FAA3E0F9E6
:10094200120C09FF900019E06F702A900001120C3E
:1009520022FF90001AE0B5071C900002120C22FF41
:1009620090001BE0B5070E900003120C22FF9000CE
:100972001CE06F60037F0022900011E0900004F001
:10098200900012E0FFA3E0900006CFF0A3EFF090FA
:100992000021E0900000F0900022E0FFA3E0900030
:0809A20002CFF0A3EFF07F018A
:0109AA00222A
:100DCD0075B283E4F5A9538EF4758920758DF97587
:0B0DDD008BFFD28E75C15D43C18022E8
:100D3F008F828E83D3E5829DE5839C5019758F0337
:100D4F0075B7A575B7F1E4F0F58F2582F5827402BA
:060D5F003583F58380DE00
:010D6500226B
:0B0B2F00900074EFF0A3EDF0A3EBF0DA
:100B3A00C2052009FDD209C200D201D203D2047F24
:100B4A0001C2C4C206D2C530C0FDE5C054F024803B
:100B5A00606224C0601A24E06003020BEE90007603
:100B6A00E0F5C2A200E43342C2C2C5E4A3F0807633
:100B7A0030C136300606D2C5C206806A30010CC2C0
:100B8A0001D202900075E0F5C2805B300211C20208
:100B9A00900074E0F5C230034DD206D2008047209F
:100BAA000044E4900077F0803D300404D2C58036DA
:100BBA00D2058032EFFD900077E0FB3395E0FAC36F
:100BCA00EB9D7480F86A98500CA3E5C2F090007708
:100BDA00E004F0D2C1900077E0B5070AC209C2C1A9
:100BEA00D2C48002D20530050853C0BF43C040C2F8
:0E0BFA0009C2C0300903020B51900078E0FFE1
:010C080022C9
:100D660090005BEFF0900065E0FEA3E0FF120E013D
:080D7600900065EEF0A3EFF020
:0A0D7E00EEFD900001E0FB120B2FC8
:010D88002248
:100DE800900004E0FFA3E0C39F500D900001E024B1
:090DF80002F0900005E004F02275
:100E01000FBF00010EC3900007E09F900006E09E17
:090E11005006120DE8E4FEFF2278
:0809AB00900058EEF0A3EFF0FC
:1009B300E490005BF0A3F0900061F0A3F090006579
:1009C300F0A3F0900002E0FFA3E0900065CFF0A356
:1009D300EFF0900000E0A3F0E490005CF090005B87
:1009E300F090000504F0E4900060F090005BE06498
:1009F3003A6025900065E0FEA3E0FF120D7E9000B3
:100A03005BEFF0900065E0FEA3E0FF120E019000A3
:100A130065EEF0A3EFF080D3900062E004F070067F
:100A2300900061E004F0900065E0FEA3E0FF120D8A
:100A33007E120D66120D1390005EEFF090006012AF
:100A43000D6A120D66120D13900063E4F0A3EFF02C
:100A5300900063A3E0FFFD900060E02DF0EF9000B5
:100A630063F0A3E4F0A3120D6E120D66120D139042
:100A73000063E0FEA3E04FFF900063EEF0FEA3EF00
:100A8300F0AC068C08F509900060E02F120D6A1295
:100A93000D66120D1390005DEFF0900060E02FF0F3
:100AA300EF706990005AF090005EE0FF90005AE00A
:100AB300C39F5058120D6B120D66120D1390005FF9
:100AC300EFF0A3E02FF0A3E0B4010AA3E0B4DA054A
:100AD300E490005BF0D3900059E09509900058E052
:100AE3009508501F758F0175B7A575B7F190005F15
:100AF300E0850982850883F0E4F58F0509E509702F
:100B030002050890005AE004F0020AAA120D6B12C3
:100B13000D66120D1390005FEFF0A3E02F700C90A1
:0B0B2300005DE0640160030209E922AC
:010B2E0022A4
:040E280002000022A2
:03000000020800F3
:03000300021A03DB
:03000B00021A06D0
:03001300021A09C5
:03001B00021A0CBA
:03002300021A0FAF
:03002B00021A12A4
:03003300021A1599
:03003B00021A188E
:03004300021A1B83
:03004B00021A1E78
:03005300021A216D
:03005B00021A2462
:03006300021A2757
:03006B00021A2A4C
:03007300021A2D41
:10080000E4F5D9E5EF7480F5FF7402F5EF787FE445
:10081000F6D8FD9000007F007E04E4F0A3DFFCDE4C
:07082000FA758121020CCAE8
:100C0900BB010689828A83E0225002E722BBFE02E9
:090C1900E32289828A83E493221C
:100C2200BB010CE58229F582E5833AF583E0225087
:100C320006E92582F8E622BBFE06E92582F8E222D1
:0D0C4200E58229F582E5833AF583E49322EB
:100C4F00BB010689828A83F0225002F722BBFE0184
:020C5F00F3227E
:100C6100A3F8E0C5F025F0F0E58215827002158346
:060C7100E0C838F0E822A3
:100C7700EB9FF5F0EA9E42F0E99D42F0EC6480C8F4
:060C870064809845F02294
:0C0C8D00ECF0A3EDF0A3EEF0A3EFF022DA
:100C9900A8828583F0D083D082120CB0120CB012D6
:100CA9000CB0120CB0E473E493A3C583C5F0C583FB
:100CB900C8C582C8F0A3C583C5F0C583C8C582C8A5
:010CC9002208
:100DAB00EF7E0024D0B40A00401624F9B40A0040A8
:100DBB000CB41000400A24E0B41000400374FFFE92
:020DCB00FF2205
:00000001FF
